:100000001CC200000C947A1B35C2000033C20000F1
:1000100031C200002FC200002DC200002BC2000020
:1000200029C2000027C200000C9451200C941D210D
:100030000C942C1A1FC200001DC200001BC200003D
:1000400019C2000017C2000015C2000013C2000050
:1000500011C200000C94A31A0DC200000BC20000D4
:1000600009C2000007C2000005C2000003C2000070
:1000700001C20000FFC10000FDC10000FBC1000083
:10008000F9C10000F7C10000F5C10000F3C1000094
:10009000F1C10000EFC10000EDC10000EBC10000A4
:1000A000E9C10000E7C10000E5C100004A001E00F0
:1000B0001F00200021002200167C380011001A00C9
:1000C0003600370050220C001800080012222F00C2
:1000D0004F211D001B0006001921302400000000E4
:1000E00034002E432A220400000000004C212B0083
:1000F0002C419124230024002500260027004D00D8
:100100000F00070005001C001300E3000A0017326F
:10011000150016000B0052322D34103109000D006D
:10012000330051310E00283231001400000000006D
:1001300090342C414B004E31000000003A003B004F
:100140003C003D003E003F00010036002400250039
:1001500026000100010055002100220023000100BB
:10016000010035001E001F002000010000000000FB
:100170000100010001002700000000000100010053
:1001800001000100400041004200430044004500DE
:100190004B004A00CD004D00DD0001004E00CF00B5
:1001A000CE00D000DE000100D300500052004F000E
:1001B000DF000100D100D200510046000000000025
:1001C00001000100025201000000000029001E0091
:1001D0001F002000210022002B00170014001A002D
:1001E00008001500E1000A000400160007000900DD
:1001F000E000E2001D001B000600190000000000E6
:1002000005001C002C000B00000000000D000E007B
:1002100018000C0023002400250026002700000001
:100220000000000052000000E50000000000500047
:1002300051004F00E6000000000000000000000038
:10024000E40000004C002C00000000000000000052
:10025000280020520052D10000000000007C010064
:100260000100010001000100010001000100010086
:100270000100010001000100010001000100010076
:100280000100010001000100010001000000000068
:100290000100010001000100000000000100010058
:1002A0000100010001003A003B003C000100010098
:1002B00001003D003E003F00010001000100400040
:1002C00041004200010001000100430044004500DC
:1002D0000100010001000100010001000000000018
:1002E0000100010001000100000000002C03440097
:1002F00061006300740079006C002D004D00610006
:100300006E00750066006F0072006D00200028000E
:10031000350078003600290000000E0374007300D9
:1003200068006F00720074000000040309040902F1
:100330003B00020100A0FA090400000103010100D2
:100340000921110100012244000705810308000171
:10035000090401000103000000092111010001222C
:100360007B0007058203200001120100020000004B
:10037000084D44363501000102000105010902A1C2
:100380000185020901A100050919012908150025A7
:100390000195087501810205010930093115812592
:1003A0007F95027508810609381581257F950175AD
:1003B000088106050C0A38021581257F950175080C
:1003C0008106C0C005010980A101850319012AB772
:1003D00000150126B700950175108100C0050C09B4
:1003E00001A101850419012AA002150126A0029588
:1003F0000175108100C005010906A101050719E07A
:1004000029E71500250195087501810295017508F8
:1004100081010507190029FF150026FF00950675C3
:1004200008810005081901290515002501950575A4
:10043000019102950175039101C011241FBECFEFF8
:10044000DAE0DEBFCDBF11E0A0E0B1E0E6EDF7E419
:1004500002C005900D92AA3AB107D9F722E0AAEAA4
:10046000B1E001C01D92A53CB207E1F70E9435132F
:100470000C947123C5CD8430C8F46C30B8F4463088
:10048000A8F450E096E0699F400D511D112498E4B6
:10049000899F400D511D1124FA01EE0FFF1FE455F5
:1004A000FF4F85919491282F822F089521E090E0AD
:1004B000FBCFE1CF089581E0089581E00895FBCF5F
:1004C000089581E0089581E00895FDCF089508958D
:1004D0000895FDCF089508950895A6E0B0E0E3E7FC
:1004E000F2E00C94E42249835A839E833091B10157
:1004F00089819A81311117C03E81311589F021150A
:1005000079F06CD5182F682F89819A8146D5698139
:100510007A81812F0E94C10D2696E3E00C9400237E
:100520004DD5182FF4CF5AD569817A81F3CFFC01CC
:10053000262F408151816281738184819581CDCF45
:10054000CF93DF93EC0161E0F2DFBE01B6DF8115EE
:1005500029F061E0CE01EBDFBE01B1DFDF91CF9189
:1005600008950F931F93CF93DF93EC0160E0DFDFDB
:100570008C01BE01ADDFBE01C801ABDFDF91CF91C1
:100580001F910F9108950F931F93CF93DF93EC0169
:1005900061E0CDDF8C01BE0194DF811106C080E0F7
:1005A000DF91CF911F910F910895BE01C8018DDF9A
:1005B0008115A9F3BE01C8010E943B18811579F38A
:1005C000BE01C8010E94B214811549F3BE01C801E1
:1005D0000E948914811519F3BE01C8010E94070FFA
:1005E0008115E9F2BE01C8010E94190F8115B9F207
:1005F000BE01C8010E94330FD3CF21E030E002C01A
:10060000220F331F8A95E2F7C90102C4CF93C82F86
:1006100081E090E00C2E02C0880F991F0A94E2F747
:100620000E94F10B8C2FE9DFCF91089581E00895AE
:1006300081E00895FBCF0895CF93C82F98D38C2FD6
:10064000F7DF8C2FF7DF8FEF94E32CE081509040A1
:100650002040E1F700C00000CF91089581E0ECDF79
:100660000C94C71A80E0E8DF0C94D81A34DF0E949B
:10067000F21917C018D030DF0C94F61981E00895F4
:100680000895CF93DF93C82FF9DFD82F811511F08C
:100690008C2FF6DF8D2FDF91CF9108950895F1CF44
:1006A000089580E0FCCF0E948018F9CFCF930E947C
:1006B0008018C82F8091AC018C1771F0C093AC01E9
:1006C0000E94971A6093AD017093AE018093AF01C1
:1006D0009093B0018C2FE3DFCF910895ADE0B0E0AF
:1006E000E4E7F3E00C94E522488759876A877B8723
:1006F0008C879D8791118ED71F8286E0FE013896E8
:100700009E012F5F3F4FD90101900D928A95E1F72D
:100710008D8181110CC029813A814B815C816D8171
:100720007E818F81C2D62D96E2E00C940123CE010A
:10073000019606DF8111EFCFF6CFFC012481213035
:1007400019F4808191817DC40895611521F00E9482
:100750000E160C94C3160E944E16FBCFCF93C82FD3
:100760008115B9F08238B9F40E94951881FD11C045
:1007700089E30E945419B7D78FEF97EE23E0815099
:1007800090402040E1F700C0000089E30E945A1920
:10079000AAD7CF910895833899F40E94951880FDC7
:1007A000F8CF83E50E9454199ED78FEF91EE24E095
:1007B000815090402040E1F700C0000083E5E6CF83
:1007C000843899F40E94951882FDE3CF87E40E9453
:1007D000541989D78FEF91EE24E08150904020404A
:1007E000E1F700C0000087E4D1CF8450813A90F453
:1007F0008C2F0E94BD138111CCCF8C2F0E94181911
:10080000811521F08C2F0E945A196DD78C2F0E94D0
:100810005419BECF8C2F805E883048F481E0C1FD32
:1008200084E0C0FD880FC2FD8295D5D6B1CF8C2F54
:10083000855A833030F48C2F8452990B0E94B6185D
:10084000A8CFEC2FE85AEB3150F4F0E0EE0FFF1F89
:10085000E15DFE4F808191810E94DD189ACF8C2F3F
:100860008D5C833108F095CF61E08C2F6EDF91CFE6
:10087000811509F44EC0823861F40E94951881FFF9
:1008800048C089E30E9454192ED789E30E945A195F
:100890002AC7833851F40E94951880FF3AC083E537
:1008A0000E94541920D783E5F1CF843851F40E9477
:1008B000951882FF2EC087E40E94541914D787E44C
:1008C000E5CF982F9450913A08F3982F905E983086
:1008D00050F4982F81E091FD84E090FD880F92FD07
:1008E00082957FD6D5CF982F955A933020F480E00B
:1008F00090E00C94B618982F985A9B3120F480E021
:1009000090E00C94DD18982F9D5C933110F460E01A
:100910001CCF08951F93CF93DF93182FEB011EDF99
:10092000209731F4812FA4DFDF91CF911F9108959B
:100930008FE99FE00197F1F700C000002197F0CF09
:1009400060E570E0893311F060E070E0E3CF81157D
:1009500011F041D6C8C60895811511F042D6C3C61C
:100960000895A0E0B0E0E7EBF4E00C94DF226C0126
:10097000D62FC72FFC011581068102950F7020D656
:10098000E82E8115E9F0E12E1115D1F08C2F807F32
:10099000803461F08D2F805E8830E0F08C2F807E77
:1009A000803221F4D230B0F00115A1F0809195028F
:1009B00082FF10C082E0B3D603D691E08927E82EEB
:1009C000EC2FE295EF70C03C78F5F0E0ED58FC4D6F
:1009D0000C94CF22E12CF4CF0C2F0F70C03110F00B
:1009E0000295007F111581F0011549F08D2F805E71
:1009F000883010F0D11105C0802FEDD574D68D2F21
:100A000040C0802FF9D5FACF8D2F32DF011561F06C
:100A10008D2F805E883010F0D11103C0802FE1D57A
:100A200002C0802FEFD55FD6E11409F4B3C0C4D55E
:100A300080FDB0C0F6011582B9D51AD2C60168D1C1
:100A4000B5D524D2A7C08C2F8F70F82EC07FC032AE
:100A500019F0F29480EFF822D13038F079F11115C5
:100A600009F438C00115C9F0CACF8091950282FD02
:100A700010C0111541F0F11419F08F2DACD533D6FB
:100A800080E06CDED1CF80E0F3DEF11469F28F2DCF
:100A9000C6CF111551F0013018F48F2D58DFC4CF97
:100AA00009F0C2CF8F2DCAD5BFCF0111BDCF8F2D79
:100AB00053DF8F2DCED58F2DB3D5B6CF111521F0A5
:100AC000063008F0B1CFE9CF053008F0ADCF8F2D5B
:100AD00043DFAACF0115D9F3D93349F48FEF97EE4D
:100AE00023E0815090402040E1F700C000008D2FAE
:100AF000BFDE9ACF8C2F869586958370813060F00B
:100B000009F092CF8D2F9C2F9370111102C080E0BD
:100B100090E00E94DD1888CF8D2F9C2F93701111CB
:100B200002C080E090E00E94B6187ECF612F8D2F2A
:100B30000CDE7ACF8C2F8370C1F5111128C04D2F98
:100B4000429546954770440F440F2D2F2F7030E08B
:100B5000042E02C0220F331F0A94E2F780E090E0D7
:100B6000D4FF09C08FE090E002C0880F991F4A951A
:100B7000E2F780959095C695C695C370822B932B0E
:100B8000C23079F0C33079F0C13049F04AD10E94C7
:100B9000801885DDCDB7DEB7E8E00C94FB223AD1B2
:100BA000F6CF46D1F4CF34D1F2CF111559F1C0FFB1
:100BB000EECF4D2F429546954770440F440F2D2F91
:100BC0002F7030E0042E02C0220F331F0A94E2F788
:100BD00080E090E0D4FF09C08FE090E002C0880F71
:100BE000991F4A95E2F780959095C695C695C37072
:100BF000822B932BC23061F0C33061F0C13031F0F1
:100C00006AD1C5CF823008F4C2CFD3CF5DD1BFCF78
:100C100069D1BDCF1AD1BBCFCF70111529F08C2F60
:100C200027D18D2F94DEB3CF8D2F96DE8C2F2ED132
:100C3000AECFD23F31F168F4D03FC1F0D13F89F05F
:100C4000111509F43EC0011509F438C08D2F86DD59
:100C50009ECFD33FE1F0D43F99F78091950282FD7A
:100C60001EC08C2F8F71111511F30FC0111539F0A3
:100C7000053008F08CCF8C2F8F7118D188CF0630BB
:100C8000F8CF8C2F8F711111D2CFF2D080CF1115E8
:100C900021F08C2F8F71E3D07ACFDED078CF111571
:100CA00029F063E08C2F8F7123D571CF81E037D588
:100CB000023008F46CCF82E032D569CF8C2F8F716F
:100CC000E4CF011571F0D93349F48FEF97EE23E0AB
:100CD000815090402040E1F700C000008D2FC8DD1A
:100CE00056CF8C2F8F71A3CF0F931F93CF93DF938A
:100CF000EC01688179818D81ADD18C01FAD087D0EA
:100D0000B801CE012EDEDF91CF911F910F91089592
:100D1000CF93DF93EC018C81811581F0CE0133DC20
:100D200081110FC04DD4811549F08D81811531F0AD
:100D30008091950282FF02C082E0F1D4DF91CF91D1
:100D40000895CE01D1DFCE010CDCF8CF80E090E039
:100D50000E94B61880E090E00E94DD185BD4C3D4F6
:100D60000E94DC160C94C3160E946019EFCF41D488
:100D7000FBCF282F92959F70963099F060F4925F88
:100D80009F70923030F4203FB1F038F481E0283E7B
:100D900038F080E008959A5FF3CF81E0243FC9F7EF
:100DA000089591E0813F09F090E081E0283E08F04D
:100DB00080E0892B089581E00895FC0124812115AC
:100DC00021F0808191813DD1D4CF80E00895A6E0CB
:100DD000B0E0EDEEF6E00C94E5222696E2E00C940D
:100DE0000123A7E0B0E0E7EFF6E00C94E5222796B8
:100DF000E2E00C9401230895FECF0895FDCF0895FD
:100E0000FADFFCDF8093D8019093D901089508950B
:100E1000F7CF08952091D8013091D901822B932BDF
:100E2000EFCF2091D8013091D90182239323E8CFCD
:100E30002091D8013091D90182279327E1CFDBCFD0
:100E40000895FDCF0895D7CF0895FDDFFADF809391
:100E5000D6019093D701089580E090E0F6CF21E08D
:100E600030E002C0220F331F8A95E2F7C901EDCFAF
:100E700021E030E002C0220F331F8A95E2F7809113
:100E8000D6019091D701822B932BDFCF21E030E068
:100E900002C0220F331F8A95E2F72095309580918A
:100EA000D6019091D70182239323CFCF21E030E068
:100EB00002C0220F331F8A95E2F78091D6019091EC
:100EC000D70182279327C1CF2091D6013091D70136
:100ED000822B932BBACF2091D6013091D701822358
:100EE0009323B3CF2091D6013091D7018227932746
:100EF000ACCF0895CF93C1E061FDC4E060FDCC0F9D
:100F000062FDC29593E0769567959A95E1F7660F35
:100F1000771F660F771F460F571FFA0140E050E01A
:100F200090E06191DF019C01042E02C03695279567
:100F30000A94E2F72695220B26272C2326272E93A8
:100F40004F5F5F4F4430510561F7CF910895A82F4F
:100F5000A77023E0969587952A95E1F7880F991F4A
:100F6000880F991F680F791FFB0140E050E080E077
:100F7000219130E00A2E02C0369527950A94E2F7B7
:100F80002170042E01C0220F0A94EAF7822B4F5FD2
:100F90005F4F4430510561F70895262F9C3068F467
:100FA000863058F4682F70E086E0989F600D711DC0
:100FB000112442EB51E0822F9DCF0895292F9C30C0
:100FC00058F4863048F490E062EB71E036E0239FFD
:100FD000800D911D1124BBCF80E00895CF92DF9248
:100FE000FF920F931F93CF93DF936C010091D60173
:100FF0001091D7018091D8019091D901082B192B1C
:10100000CFE0D0E081E090E00C2E02C0880F991F65
:101010000A94E2F780239123892B61F4219790F7BA
:10102000F12C8F2DDF91CF911F910F91FF90DF90C9
:10103000CF900895FC2EB6018C2FAED5019771F399
:10104000F0CFCF93DF93EC01C9DFBE01A5D5DF91CF
:10105000CF9108950F931F93CF938B019091B1017E
:10106000911531F0CB01EDDFCF911F910F910895D4
:10107000811551F0CB01B2DFC82F682FC8018DDF79
:10108000B8018C2F89D5F0CFCB0198DFC82FF8CFCE
:101090000F931F930091DA018091DB01801303C04D
:1010A0001F910F91089587E0089FF0011124E452E9
:1010B000FE4F208131814281538164817581868117
:1010C00090DE0F5F1F4F0770E7CF20911402309121
:1010D000150240911602509117026091180270910A
:1010E000190280911A027DCE80911A02803170F42B
:1010F00080911902811551F0E091DA012091DB0114
:1011000030911502409114022E1301C00895BF01C1
:1011100087E0E89FF0011124DF01A452BE4F14962E
:101120008C911497811549F111968C911197831325
:1011300024C08C91841321C015968C911597811130
:101140001CC012968D919D91A0911602B09117022C
:101150008A1B9B0B883C910580F480911A028F704A
:10116000806180931A02EE51FE4F80818F70806102
:10117000808384E192E0CCDD8BCF6F5F7F4FFB01FA
:10118000E770C2CF8F929F92AF92BF92DF92EF92A1
:10119000FF920F931F93CF93DF93CDB7DEB72D97B9
:1011A0000FB6F894DEBF0FBECDBF8C0186E0F8010C
:1011B000DE01189601900D928A95E1F7F801F5800D
:1011C000848194E1892E92E0992E909118029111D8
:1011D00017C0811509F416C1F11409F455C1C801ED
:1011E000ECDD811509F450C187E0F801D4010190CC
:1011F0000D928A95E1F7C401A0DA76DF66DF02C1BD
:101200007081A280B380D090190220911602309193
:101210001702A501421B530BD11409F4F6C0483C38
:10122000510508F0C5C0811509F4ECC030911502D4
:10123000218180911A02803108F08CC0EF2C231399
:1012400026C030911402371322C0F11027C08F70CE
:10125000806180931A0239DF84E192E059DD809148
:101260001A02F8018683E12C8E2D2D960FB6F89484
:10127000DEBF0FBECDBFDF91CF911F910F91FF90C9
:10128000EF90DF90BF90AF909F908F9008958091E6
:10129000DA013091DB01E82FF114D1F080911A02CC
:1012A000816080931A02DFCFAF0167E06E9FF0018B
:1012B0001124E452FE4F6181261306C0608176132B
:1012C00003C065816111EBC04F5F5F4FFA01E770AA
:1012D000E313EACF381310C088859985B2DE292F31
:1012E00022952F709034E0F02A5F2F70223060F149
:1012F000C8010EDDED2CB8CFAC0167E0869FF00190
:101300001124E452FE4F8181281306C08081781396
:1013100003C085818111A7CF4395842F8770DACFD1
:101320009F70223038F0911551F0F801968190317C
:1013300030F49ACF911519F0811509F495CF805E9C
:10134000883008F491CFD4CF803F08F48DCF815FEF
:101350008330F7CF231307C020911402271303C053
:10136000F11409F473C0C80128DD811509F48CC09B
:10137000F11409F489C080911A02803280F0209122
:1013800014023091150229833A83AB82BC8290917A
:1013900018029D831E828F83CE010196B9DC87E0FF
:1013A000F801A4E1B2E001900D928A95E1F725CF12
:1013B00020911A02203188F4488559856A857B85F9
:1013C0008C859D8504DD84E192E0A2DCF40187E058
:1013D00011928A95E9F779DE46CF811599F030911F
:1013E000150281813813BFCF809114028713BBCFC0
:1013F000F110B9CF2683C8018BDCF40187E011928C
:101400008A95E9F7EE24E3942FCF483C510508F084
:101410003EC08115B9F3F114B9F120911502818113
:10142000281329C080911402871325C080911A02C5
:1014300080FD18C08031B0F08683807F803F39F016
:101440008681982F907F905F8F70892B8683C8014B
:101450005FDC87E0F801A4E1B2E001900D928A958B
:10146000E1F7CCCE87E0F801A4E1B2E001900D9263
:101470008A95E1F7C7CFC801A0DC811190CF809198
:101480001A02816080931A02C80142DCBBCF4885F2
:1014900059856A857B858C859D8599DC97CF84E10C
:1014A00092E036DCE4E1F2E092CFAEE0B0E0EBE5D2
:1014B000FAE00C94E422288739874A875B876C8797
:1014C0007D878E87CE0108965DDE6C85811599F04B
:1014D000611539F0288539854A855B857D858E853E
:1014E00080DC8091DA019091DB0189133DC02E965A
:1014F000E3E00C94002387E09E01285F3F4FF90151
:1015000027503109D90101900D928A95E1F76115B3
:1015100041F3A091DB018A2F90E08395877090E0E2
:10152000AC012091DA012417150691F097E09A9FFB
:10153000D0011124A452BE4F9E012F5F3F4FF901ED
:1015400001900D929A95E1F74093DB01A1DDC9CF9F
:101550000EDC1092DB011092DA01E4E1F2E087E0A8
:1015600011928A95E9F7BDCF17E0189FC0011124A9
:1015700084529E4F07DE811509F4B9CFE091DA015C
:101580001E9FF0011124E452FE4F208131814281DF
:10159000538164817581868124DC8091DA01909188
:1015A000DB01019687708093DA019BCF8091230243
:1015B0008695869586950895809123028770089573
:1015C00090912302977081E0911101C080E008950D
:1015D00080912F02089590912F02982B90932F02C3
:1015E00008958095982F80912F02892380932F0250
:1015F000089510922F02089590912E02982B9093A7
:101600002E0208958095982F80912E028923809331
:101610002E02089510922E0208950895FECF089587
:1016200090912402292F282329F0809589238093E3
:101630002402F4CF08950895FECF089590912502D5
:10164000292F2823281721F0982B90932502F4CFD7
:10165000089590912502292F282329F08095892328
:1016600080932502E9CF089580912502811521F00C
:101670001092250280E0E0CF08950F931F93CF933F
:10168000DF9380910001909101018C01C0912F02A4
:1016900080912E02C82B80912502811529F0C82B3C
:1016A0000E9404198111E0DFF801C083C09100019C
:1016B000D091010148E050E06BE172E0CE010E9460
:1016C0002023892B59F088E0FE01ABE1B2E00190C4
:1016D0000D928A95E1F7CE010E949718DF91CF9184
:1016E0001F910F910895C9CF08950895FECF0895D1
:1016F0009091950292FF0EC0982F990F990F990F14
:10170000962B90932302B4DB8091230286958695D5
:101710008695ECCFADCB1092230280E0E7CF90917D
:1017200023028095892380932302282F277059F460
:10173000891749F09091950292FF05C0869586958C
:101740008695A4DBE8CF08959091950292FB22271D
:1017500020F9281749F080FB92F99093950284E9CB
:1017600092E043D082E0DBCF08958091950200247F
:1017700082FF0394802DE8CF81E0E6CF80E0E4CFC4
:1017800080E090E0BC01D6C380E090E0BC01CCD307
:10179000F7CFA3E0B0E0EFECFBE00C94E5227DD3C3
:1017A00088D31B82CE0103969BD381E090E0809387
:1017B000D8011092D901A0D3198284E18A83CE0185
:1017C0000196ABD3E1DF2396E2E00C940123E1CF55
:1017D000089575C3089562C3089577C3089586C3B5
:1017E00008958AC308958DC3089597C30895A8C323
:1017F0000895B0C30895A6E0B0E0E1E0FCE00C94E9
:10180000E3220E948B1A8C01809130029091310268
:101810008017910779F019821A820E948B1ABC01F5
:1018200049815A8180E090E00E946E03009330026B
:10183000109331022696E4E00C94FF22CAD2609302
:101840004202709343028093440290934502609356
:101850003E0270933F0280934002909341020895AC
:1018600008950895FDCF08950895FEDFFBCF0895F4
:10187000FECF08950895FEDFFBCF81E0089585E057
:101880009FE003D7EEDFF1CF1AC5089508950895BC
:101890000895FCDFFCDFFCCF9EDF811101C097DFE4
:1018A00086E492E09ADF84E992E09DDF98DFB0DA87
:1018B0008091D6019091D701C4CA0E94821A60D249
:1018C00001D543D4E9DF0E944E030E946F1407D56F
:1018D000D2CFA6E0B0E0EFE6FCE00C94DD22CDDF55
:1018E00081110AC088DFEBD40E94FD160E945603C6
:1018F0002696EAE00C94F92246D482E3A82E82E0F0
:10190000B82E750110E0F7010081812F2ED31F5FE3
:101910001C3009F43EC09FEFE91AF90A081799F341
:101920008091460281FD27D3AFDFC82E10E0812FC2
:101930001CD3082FF50181915F01081729F1802739
:10194000D82EEE24E394F12C8E2D8D21B1F0C1140C
:10195000A1F0F9821A830E948B1A8B839C8381E009
:101960008D8391E08E2D802309F490E049815A8186
:101970006B817C818D810E946E03F394EE0C8F2D20
:10198000863011F7F50102931F5F1C3081F656DF98
:10199000AACF0813C5CFA6CF0F931F93CF93DF9382
:1019A000FDD0EC01D23508F050C0D03508F0C8C0E9
:1019B000C03ED10530F5CD3CD10508F09DC0C83AF8
:1019C000D10578F4C53AD10508F093C0C130D105EE
:1019D000B1F1CE010497813A910588F1C0E0D0E0E1
:1019E0002EC0CE01885A91094B97C0F7C85AD0E053
:1019F000CC0FDD1FCB59DE4F0990D881C02DD464A8
:101A00001EC0D034A8F4D03208F0ADC0C83ED10515
:101A1000B0F0CE0191509F3108F78D2F62D1082F81
:101A20008C2F90E0BBD0D02FDF71C82FD92B07C0EF
:101A30008C2F90E0B3D0DF70C82FD92BD06ACE01A5
:101A4000DF91CF911F910F910895C03882E5D8079B
:101A5000B8F5C03682E5D80708F056C0C03482E534
:101A6000D807C8F4C03282E5D80708F047C08C2FE9
:101A70008695869520E2829FC0011124C37021E0E3
:101A800030E002C0220F331FCA95E2F7E901C82BEC
:101A9000D92BDD68D4CF8C2F86958695877020E270
:101AA000829FC0011124C37021E030E002C0220FE8
:101AB000331FCA95E2F7E901C82BD92BDC68BFCFE9
:101AC000C03C82E5D80750F48C2F8F71C03AD245C4
:101AD00080F5982F84EF906AEC01B1CFCE01805C45
:101AE0009245809708F07ACFDC2FDF71C0EFD06A83
:101AF000A6CFA497D064A3CFD065A1CF8C2F8F7130
:101B0000D82FC1EFD06A9BCF8C2F86958695877092
:101B100020E2829FC0011124C37021E030E002C0A6
:101B2000220F331FCA95E2F7E901C82BD92BDA68D7
:101B300086CFD7D0982F80E09F71EC01D0627FCF05
:101B40008C2F8F71CED053E0CC0FDD1F5A95E1F76B
:101B5000DF70282F84FF04C090E1899F9001112439
:101B6000C22FD0696CCF8D2F8F71BBD0082F8C2FD7
:101B700090E014D0302F3F71282F392B3062E901CB
:101B80005ECF462F7C3028F4663018F4672F0C9413
:101B9000590280E090E00895F4DFFECE803E91058A
:101BA000D1F1C8F48133910509F481C048F4893238
:101BB000910509F471C08A32910509F47FC0089536
:101BC00089339105E1F082389105C9F0853391059B
:101BD00009F45DC00895843E9105D1F148F4823E38
:101BE000910531F1833E910541F181EE90E0089538
:101BF000863E9105C1F1873E9105F1F1089520914E
:101C00009402237009F064C02091950223FF14C050
:101C100089E290E008952091940220FD45C0309122
:101C2000950230FF09C024FD24C083EE90E00895A2
:101C30002091940222FDF7CF08952091940222FD75
:101C400044C03091950230FD43C024FFF5CF11C050
:101C50002091950221FFF0CF8091940284FD09C06C
:101C600087EE90E008952091940223FFE5CF24FFB2
:101C7000F7CF80E090E008952091940223FD2BC0DF
:101C80003091950231FFE1CF84EE90E008952091EC
:101C9000940225FFD1CFBCCF2091940225FD1EC018
:101CA0002091950223FFC8CF89E390E00895209109
:101CB000940226FFC1CF8AE290E008952091940219
:101CC00026FFBACF81E390E0089582EE90E0089578
:101CD00080EE90E0089586EE90E0089585E390E030
:101CE00008959091940292FF10C041E0282F247132
:101CF000243009F040E031E0282F2871283009F025
:101D000030E0431711F02CE0822793FF10C041E030
:101D1000282F2471243109F040E031E0282F287168
:101D2000283109F030E0431711F02CE08227309180
:101D3000950230FF10C051E0282F2171213009F0A9
:101D400050E041E0282F2871283009F040E0541776
:101D500011F029E0822731FF10C041E0282F2171C6
:101D6000213109F040E031E0282F2871283109F0B5
:101D700030E0431711F029E0822794FD877E089513
:101D80001092960210929702109298021092990265
:101D90000895EF92FF920F931F937B018C018FD2D6
:101DA000811112C00E94971A9701A801261B370BB8
:101DB000480B590BC901DA01809396029093970260
:101DC000A0939802B09399021F910F91FF90EF900A
:101DD000089575D2811541F00E94971A462F572F0A
:101DE000BC01CB01BA0108950E94971ADC01CB0116
:101DF00040919602509197026091980270919902D9
:101E0000480F591F6A1F7B1FECCF80E00895CF93C6
:101E10009C01205E3245C1E02032310538F4FB01DF
:101E2000C581C11103C08F710E9406038C2FCF9111
:101E300008959C01FB018581811599F02B359CE764
:101E4000390769F02C359CE7390721F02A353C47E2
:101E500021F008958ADC80E008958EDCFCCF8EDCD2
:101E6000FACF81E008959C01FB018581811599F0ED
:101E700021309CE7390761F023309CE7390739F0BE
:101E800021153C4749F40E942E0380E00895A1DC0F
:101E90000E943203FACF81E00895089580E090E037
:101EA0000E943E239C0181E0233E3E4F09F080E0EA
:101EB000089563EE7EEF80E090E00C945D236FEF79
:101EC0007FEF80E090E00C945D23CF93DF93EC01F3
:101ED00082E090E00E9436238883DF91CF910895BD
:101EE000FC01608182E090E00C94432383E090E069
:101EF0000E94362390E00895682F83E090E00C94D0
:101F00004323CF93DF93EC0184E090E00E943E23D3
:101F100088839983DF91CF910895FC01608171815D
:101F200084E090E00C945D23AB01BC018FE090E075
:101F30000C945523AB01BC0183E190E00C94552334
:101F40008EE090E00E943623982F81E0911101C02D
:101F500080E00895682F8EE090E00C94432308956C
:101F6000FECF08950895FECF0895E82FF0E0E955DB
:101F7000FD4F80810895089580EA8A95F1F70895CC
:101F800000C00895F9CF08950895FECF0895A6E002
:101F9000B0E0EDECFFE00C94E02291D1F82E8091BE
:101FA000B30290E089559D4FF114E1F18E010F5F6E
:101FB0001F4FF80126E011922A95E9F7B8019BD14D
:101FC000E02ED12E8115B1F080919A0290E046E08A
:101FD00050E0B80189559D4F0E94202321E02093B5
:101FE0004702892B91F4F12CBEDF8F2D2696E7E076
:101FF0000C94FC22809147028115A9F3F80186E038
:1020000011928A95E9F710924702A0919A02B0E0E6
:10201000A955BD4F86E0EE2DFD2D01900D928A95BC
:10202000E1F7E2CF20919A0230E0BC01C901895565
:102030009D4FECD1AADFD9CFF894E82FE295EF704D
:10204000F0E041A18F7021E001C0220F8A95EAF7EC
:10205000922F9095942391A392A1822F892B82A3F2
:1020600078940895CF93DF93C1EAD1E089918F3FAF
:1020700009F0E2DF81E0C73AD807C1F7CBE9D1E048
:1020800089918F3F09F0D8DF81E0C13AD807C1F7C5
:10209000DF91CF910895A0E0B0E0E1E5F0E10C948C
:1020A000DF226C01E62EC62FD0E08E010F551E4FA9
:1020B000F80180818F3F09F441C0F894E82FE29540
:1020C000EF70F0E091A18F7021E001C0220F8A959E
:1020D000EAF7892F822B81A382A12095282322A3AE
:1020E00078944EDFABE9B1E031E0F12C2D912F3F38
:1020F00079F0E22FE295EF70E05EF0E0808190E011
:102100002F7002C0959587952A95E2F780FF1BC036
:1021100080E0F82A330F81E0A13AB80739F7F801D7
:1021200080818F3F09F088DF61E0F11001C060E03D
:102130008E2D28DFF601EC0FFD1FF082CDB7DEB744
:10214000E8E00C94FB22832FE4CF80910201809180
:10215000020190E0811101C096E09093B30286E005
:10216000891B80939A027EDFE7EAF2E08CE011920D
:102170008A95E9F7EBE9F2E08CE011928A95E9F7AC
:1021800086E042D0EDCEACE0B0E0E9ECF0E10C94BA
:10219000E222FE013196DF018CE01D928A95E9F77B
:1021A00010E00E2FFF2E612F802F9F2D74DF812FC7
:1021B0008F5F182F8630B9F74CE050E0602F7F2DED
:1021C0008BE992E00E94202321E0892B99F420E002
:1021D0006091B30270E069557D4F46E08BE992E073
:1021E00014D0182FD4DE912F982B892F2C96E5E050
:1021F0000C94FE228CE0E02FFF2DABE9B2E00190C1
:102200000D928A95E1F7E4CF0895A0E0B0E0EBE00D
:10221000F1E10C94DF227C016B01042FC22F211508
:1022200079F081E080934A020E948B1A80934802E1
:102230009093490280E0CDB7DEB7E8E00C94FB2232
:10224000D0914A02D115B1F3809148029091490290
:102250000E940A1A059770F310E0A801B701C601A1
:102260000E942023892B31F0A801B701C6010E94EA
:102270002D23CD2F10924A028C2FDDCFACDA8111A5
:1022800001C0A5DAB4CA1F93CF93DF93C8ECD0E0A6
:102290000E94B622182F81110AC08FE39CE9019792
:1022A000F1F700C00000219799F70E94B222812F18
:1022B000DF91CF911F91089580914E0208958091F2
:1022C0004D020895E0DF80934D02D8DF80934E02E7
:1022D000F3DF80930201F3DF811140C00895EFDF47
:1022E000811101C03EC0089581E090914F029A3063
:1022F00008F080E008950F931F93CF93DF93EC01D4
:102300008B0180914F028A3080F4B801CE017CD0DD
:10231000811121C080914F028F3FB1F40E948B1A2E
:1023200080934B0290934C0209C080914B02909194
:102330004C020E940A1A843F914038F780E0DF91F6
:10234000CF911F910F9108958F5F80934F028A3034
:1023500028F781E0F4CF10924F02FBCF0C94361B8C
:1023600008950C94391B0895CF92DF92FF920F933A
:102370001F93CF93DF936901E801082F880F110B9A
:1023800041155105B1F0F80133E0EE0FFF1F3A950A
:10239000E1F7ED5FFE4F81819281805B9D4FE0818F
:1023A0002E2F30E04E17510508F49A01A9010E9422
:1023B0002D23C8010E94171CF82E8115E1F02097EB
:1023C000D1F0C80123E0880F991F2A95E1F7FC019D
:1023D000ED5FFE4F2381422F50E0C217D10508F474
:1023E000AE018D5F9E4FFC0164817581605B7D4F06
:1023F000C6010E942D238F2DDF91CF911F910F9148
:10240000FF90DF90CF900895E7C00895FAC0089537
:10241000A4E0B0E0EEE0F2E10C94E3226091690206
:1024200070916A0280916B0290916C02FCD711E06E
:10243000643671058105910508F1CBDCDC01CB0127
:102440000296A11DB11D89839A83AB83BC8300E0F2
:1024500010E0980144E050E0CE010196BC0182E01A
:1024600083DF182F811551F00E94971A609369023B
:1024700070936A0280936B0290936C02812F249672
:10248000E4E00C94FF22A7E0B0E0E9E4F2E10C9470
:10249000DD225B01E090A701F090A80101E010E0CF
:1024A000CE0107969C0140E050E0BA0180E05CDF7D
:1024B000182F811509F444C067018FEFC81AD80A94
:1024C0006091650270916602809167029091680246
:1024D000AAD7643671058105910558F106E010E030
:1024E000CE0101969C0140E050E0BA0181E03CDF62
:1024F000182F66E070E0C601F3D19F8198132DC0BC
:10250000111559F10E94971A609365027093660243
:10251000809367029093680286E09E012F5F3F4F91
:10252000F901AFE5B2E001900D928A95E1F781E003
:1025300015C066E070E0C601D3D19F818913CECF6C
:1025400086E0F70131969E012F5F3F4FD901019040
:102550000D928A95E1F71111DFCF80E096E0EFE56B
:10256000F2E0D50101900D929A95E1F72796EAE005
:102570000C94F922A0E0B0E0E0ECF2E10C94DD2252
:102580007C016B015A01B0DE0AE010E0811102C04B
:1025900001E010E0C1E0D0E0B601C701F501099506
:1025A000811115C021960C171D078CF0CC9F90014E
:1025B000CD9F300D300D112480E090E045E34A9529
:1025C000F1F70000019682179307C1F7E5CFCDB769
:1025D000DEB7EAE00C94F9220F931F93CF93DF93B9
:1025E000EC018B0143E452E1C5DF811529F048E09D
:1025F00052E1B801CE01BEDFDF91CF911F910F9163
:102600000895CF93DF93C091A701D091A801CE0187
:10261000019626E0FB01DC0101900D922A95E1F77D
:1026200066E070E05DD188838F819885A985BA8541
:1026300040915B0250915C0260915D0270915E027C
:1026400084179507A607B70759F080935B0290930C
:102650005C02A0935D02B0935E02BC01CD0199DBE8
:10266000DF91CF91089535C90895EFD60E94A71D37
:1026700006D90E94BF1D21D90E94C81D0E94CB1DF2
:10268000F2DF0E94EA1D05D9F9CF8093AA01909349
:10269000AB0108958B3258F4853098F0E82FE5505F
:1026A000E63278F4F0E0E158FC4D0C94CF2283340C
:1026B00050F48A3308F051C0853331F091E088330B
:1026C00061F090E00AC0E9F781E090E00E9408071D
:1026D0000E94B70601C07BD891E0892F08958091B0
:1026E0004602807F8093460281E080937002F4CF9F
:1026F0000E942E03F1CF90914602892F8E7F90FF8A
:1027000081608093460280FDE7CF817F80934602FF
:10271000E3CF90914602892F8D7F91FF8260809355
:10272000460281FFD9CF809146028160EFCF909120
:102730004602892F8B7F92FF84608093460282FD40
:10274000F2CFCACF90914602892F877F93FF88608E
:102750008093460283FDE7CFBFCF895321E030E06D
:1027600002C0220F331F8A95E2F7C901AFCF8D5106
:10277000F5CF80E0089580E00895CF93C82F809131
:102780007002813089F0823081F18111A4C00E94F1
:10279000E80A823209F0A1C08C2FEBDF811102C060
:1027A0008C2F78DFCF9108950E94E80A8232A1F33E
:1027B0008C2FE1DF811519F081E08170F3CFC431F6
:1027C00069F030F4CB30C1F3C03159F080E0F5CF7F
:1027D000C93221F081E0C833C9F7EFCF10927002FF
:1027E000F5CF82E080937002E7CFCF3409F469C05F
:1027F00068F4C83248F4CE3178F5C73009F450C0D7
:10280000C431F9F081E0CECFC932FBCFC13509F434
:102810005AC0C23509F459C086EFC03599F7E09126
:102820006D02F0916E02309769F32081982F990F15
:10283000990B820F911D91300CF449C08FEF80836A
:10284000E1CF80916F028115E9F210926F02109230
:102850006D0210926E02D6CFCD51C0936F02C4307C
:10286000C9F078F480E291E0C23031F083E792E081
:10287000C33011F48FE191E080936D0290936E026A
:10288000C1CFC53051F08BE191E0C630A9F3109271
:102890006F02B8CF8EE191E0EFCF8CE191E0ECCF09
:1028A0001092730284E180932001C0931F018CE396
:1028B00080931E0188E080931C0188E280931B01B5
:1028C000A1CF8AE0ACCF8FEFAACF81E0A8CF97FF4E
:1028D000B6CF108297CF1092700280E063CF089538
:1028E000FC01680F791F8FEF41E3E617F70709F442
:1028F00008959191892728E030E0982F990F87FF5C
:1029000006C0892F842721503040B9F7EECF892F98
:10291000FACFCF93DF93EB0186319C4709F50E94F4
:10292000E80A9D81911599F08A7A91E0811101C0A0
:1029300090E090937102811541F085E3B5D40E9437
:10294000730B80E0DF91CF91089589E2F7CF8091FA
:102950007102811519F085E3ADD4F1CF89E2FCCF86
:1029600081E0F0CFCF93DF93EC01FB0185818115EE
:1029700009F4CBC09E0130572332310508F0ABC0BB
:1029800084E992E00E94F30BFE01E150F047E2324D
:10299000F10520F4EB55FC4D0C94CF22809194026C
:1029A00081608093940290C08091950288608093AA
:1029B00095028AC0809194028260F3CF8091940244
:1029C0008460EFCF809194028860EBCF8091950274
:1029D0008160EDCF809195028260E9CF8091940271
:1029E0008061DFCF809194028062DBCF809194027E
:1029F0008064D7CF0E94B706809194028068D1CFBF
:102A0000809194028C60CDCF809195028360CFCF6E
:102A1000809194028E7FC5CF80919502877FC7CF2A
:102A2000809194028D7FBDCF809194028B7FB9CF2E
:102A300080919402877FB5CF809195028E7FB7CF2A
:102A4000809195028D7FB3CF809194028F7EA9CF24
:102A5000809194028F7DA5CF809194028F7BA1CF2E
:102A60000E94B706809194028F779BCF8091940249
:102A7000837F97CF809195028C7F99CF909194021C
:102A8000892F8B7F92FF8460877F92FF886089CF38
:102A900080919502982F909590FB80F990FB81F999
:102AA00086CF90919402892F8F7B96FF806479CF97
:102AB0000E94B70690919402892F97FB87F980585E
:102AC00070CF81E00E94F90B84E992E00E94F50B3F
:102AD0000E94B70680E0DF91CF91089580E0F2CFA9
:102AE00090919402892F8F7E94FF80615ACF9091AC
:102AF0009402892F8E7F90FF816053CF9091950231
:102B0000892F877F93FF886052CF81E0E4CF382FF1
:102B100025EB3203C001112497FF04C080589109AE
:102B2000892F089580589F4FFBCF80917A0280FFB4
:102B30000DC060911F0170E0660F771F603871054E
:102B400088F56115710581F1862F089581FF07C011
:102B500060911F0184E0689FB0011124EFCF82FFD4
:102B600004C060911F0188E0F6CF90917902911521
:102B7000B9F060911E0180911F01961728F098E02E
:102B8000899FB0011124DACF899FC001112423E06D
:102B9000880F991F2A95E1F770E00E94BC22CECFE2
:102BA00068E0D2CF8FE7089581E0089580917A029E
:102BB00080FF0CC060911C0170E07595679575955C
:102BC00067956115710541F1862F089581FF06C053
:102BD00060911C0170E075956795F3CF60911C01C1
:102BE00082FD0BC0909178029115A1F060911B01BC
:102BF00080911C01961738F0682F70E060387105DD
:102C000000F38FE70895899FC001112470E00E94AE
:102C1000BC22F4CF61E0D8CF81E00895E82FED5CCD
:102C2000E33198F5F0E0E953FC4D0C94CF227DDFC1
:102C3000819580937E02089578DFFBCF76DF8195C2
:102C400080937D02089571DFFBCFB0DF80937F0218
:102C50000895ACDF8195FACFA9DF8195809380023A
:102C60000895A4DFFBCF815D990B21E001C0220F05
:102C70008A95EAF780917C02822B80937C020895EA
:102C800080917A02816080937A02089580917A021D
:102C90008260F9CF80917A028460F5CF40917D0205
:102CA0008D3C59F480917E0287FF0DC010927E0208
:102CB000411559F41092790208C08E3C81F480913C
:102CC0007E0218169CF3411581F080917F0290914D
:102CD0008002892B09F056C01092780208958F3C2B
:102CE00041F447FFF0CF10927D0280917E02811562
:102CF000E0CF803D19F41416B4F3E5CF90917F0234
:102D0000893D29F41916FCF610927F02DCCF8A3D2A
:102D100019F497FFD8CFF8CF909180028B3D29F41A
:102D200097FFD1CF10928002CECF8C3D19F41916A7
:102D3000CCF3C9CF982F915D983078F4815D990BD1
:102D400021E001C0220F8A95EAF7822F80959091A9
:102D50007C02892380937C02B6CF8D3D31F4809133
:102D60007A028E7F80937A02AECF8E3D21F48091DD
:102D70007A028D7FF7CF8F3D09F0A5CF80917A023F
:102D80008B7FF0CF0895C7D39C0190917D028091F5
:102D90007E02982B21F02093760230937702909157
:102DA0007F0280918002982B21F02093740230934F
:102DB00075028BE792E0C8C1EBE7F2E086E0119282
:102DC0008A95E9F7109279021092780210927A02AD
:102DD0000895FC01828181110EC0838181110BC095
:102DE0008481811108C091E08581811101C090E04A
:102DF000892F8170089581E0FCCFA6E0B0E0E3E088
:102E0000F7E10C94E22286E0EBE7F2E09E012F5F0F
:102E10003F4FD90101900D928A95E1F710927D0202
:102E200010927E0210927F02109280028B819C8110
:102E3000892B022FF32E811581F0809176029091DB
:102E40007702E8D2AC01909179029115A1F18091BD
:102E500020018417150608F43BC08D819E81892BC3
:102E600089F08091740290917502D4D2AC01909156
:102E70007802911509F45AC080911D018417150636
:102E800008F462C0602F7F2D8BE792E023D281117E
:102E900004C08BE792E09DDF811175DF86E0E02FB3
:102EA000FF2DABE7B2E001900D928A95E1F72696EF
:102EB000E5E00C94FE22209173028AE0289F9001A5
:102EC00011242417350748F69F5F9093790202C0BA
:102ED0009F3FD1F71B81111551F027DE91E01116AC
:102EE0000CF09FEF899F802D112480937D021C811F
:102EF000111551F01ADE91E011160CF09FEF899F29
:102F0000802D112480937E0280917D02811509F429
:102F1000A4CF10917E02111509F49FCFF8DD8093A4
:102F20007D02812FF4DD80937E0297CF2091720283
:102F30008AE0289F900111242417350708F0A2CFBA
:102F40009F5F9093780202C09F3FD1F71D811115BA
:102F500051F02CDE91E011160CF09FEF899F802D2F
:102F6000112480937F028E81182F811551F01EDE6F
:102F700091E011160CF09FEF899F802D1124809312
:102F8000800280917F02811509F47CCF90918002AC
:102F9000192F911509F476CFBADD80937F02812F26
:102FA000B6DD809380026ECF0F931F93CF93DF9394
:102FB000C42FD22FFC0185818115C9F04093830273
:102FC000AAD280938102909382028C2F805E8830F7
:102FD00048F481E0C1FD84E0C0FD880FC2FD829508
:102FE0000E94A704DF91CF911F910F910895109136
:102FF0008302141333C080918102909182020AD21D
:10300000883C910558F5CD2FC05E1D17C1F0812F6A
:10301000805E883048F481E011FD84E010FD880F67
:1030200012FD82950E94AC04C83048F481E0D1FDC5
:1030300084E0D0FD880FD2FD82950E94A704802FE6
:103040000E94A00481E0D1FD84E0D0FD880FD2FD74
:103050008295C83038F60E94AC04C4CF8C2F805EB5
:10306000883008F0BFCF81E0C1FD84E0C0FD880F4B
:10307000C2FD8295F0CF0F93FC01CB01E851FC47D4
:10308000E730F10588F5E652FC4D0C94CF2206E2BC
:1030900021EE41EE6AE17CE787DF80E00F91089541
:1030A00007E225EE45EE6BE17CE7F6CF06E221EE86
:1030B00040EE68E17CE7F0CF07E225EE44EE69E1FF
:1030C0007CE7EACF06E221EE42EE6CE17CE7E4CF5A
:1030D00007E225EE46EE6DE17CE7DECF08E221E077
:1030E00045EE6EE17CE7D8CFFB018581811110921E
:1030F000830281E0D3CF8093890290938A0208955E
:10310000DED8811103C0809184020895E091890284
:10311000F0918A02309739F00190F081E02D3097DC
:1031200011F00995089580E00895EACF0895E0919F
:103130008902F0918A02309731F00280F381E02D0C
:10314000309709F009950895E0918902F0918A027B
:10315000309759F026813781232B39F022E0DC01AA
:103160002C930680F781E02D09950895A3E0B0E047
:10317000ECEBF8E10C94E522209187023091880273
:1031800028173907B1F08093870290938802E09165
:103190008902F0918A02309761F00084F185E02D78
:1031A000309739F023E029838A839B83CE010196EF
:1031B00009952396E2E00C940123A3E0B0E0E3EE4E
:1031C000F8E10C94E52220918502309186022817BF
:1031D0003907B1F08093850290938602E0918902CD
:1031E000F0918A02309761F00084F185E02D3097EC
:1031F00039F024E029838A839B83CE0101960995C7
:103200002396E2E00C9401234091000150910101CA
:103210009A012E5F3F4F485F5F4F80E0F901908138
:103220002F5F3F4F91118F5F42175307B9F70895F2
:10323000811591F02091000130910101F901329640
:10324000285F3F4F9081981731F03196E217F307CE
:10325000C9F780E0089581E008959C01FC01329651
:1032600080E09FEF4081461759F031969F3F19F457
:10327000411101C0982F8F5F8630A1F79F3F09F45D
:103280000895290F311D97FD3A95F901628308953C
:10329000FC01329608962191261302C0DF011E928E
:1032A000E817F907C1F70895682F80910001909100
:1032B0000101D3CF682F8091000190910101E8CFE7
:1032C000E0910001F0910101329686E011928A9519
:1032D000E9F70895DC01FB0111969C91119781811A
:1032E000981322C012968C911297811519F0928131
:1032F00089131AC013968C911397811519F0938135
:10330000891312C015968C911597811519F0958126
:1033100089130AC014969C91911521F081E02481B3
:10332000291303C080E001C081E0817008950895F1
:10333000FECF08958F5F80932401609121017091E9
:1033400022018091230190912401F2CF83E08093A8
:1033500024016091210170912201809123019091BB
:103360002401E6CFE7CF089581E0809324016091A6
:103370002101709122018091230190912401D8CFE5
:10338000F3CF089591E0811101C090E09093230163
:10339000609121017091220180912301909124017B
:1033A000C7CF80912301089580932201609121016C
:1033B000709122018091230190912401B9CF8091D5
:1033C00022010895809321016091210170912201D1
:1033D0008091230190912401ABCF80912101089528
:1033E00008950895FECF089508950895F9CF08959A
:1033F000CF93FADF0E94C310F8DFC0E08C2F0E9449
:10340000B50F811105C0CF5FCC30C1F7CF910895C2
:1034100081E0FCCFCF93DF93EC017DD08C1B9D0B23
:10342000DF91CF910895EF92FF920F931F937B014D
:103430008C017DD09701A801621B730B840B950B47
:103440001F910F91FF90EF90089585B7806885BF19
:1034500085B7806885BF08951F921FB61F921124FB
:103460008F939F93AF93BF9380918B02811113C071
:103470008091B4029091B502A091B602B091B702CA
:103480004196A11DB11D8093B4029093B502A09303
:10349000B602B093B702BF91AF919F918F911F90E9
:1034A0001FBE1F9018958091BC02843031F10E949C
:1034B000360310928B0288E190E020E40FB6F89476
:1034C000A895809360000FBE2093600083B7817F32
:1034D000846083BF83B7816083BF7894889583B706
:1034E0008E7F83BF0FB6F894A895809160008861A5
:1034F00080936000109260000FBE08950E94B7068E
:103500000C943A0382E084BD93E095BD9AEF97BD99
:1035100080936E0008952FB7F8948091B402909133
:10352000B502A091B602B091B7022FBF08952FB790
:10353000F8946091B4027091B5028091B6029091B6
:10354000B7022FBF089578941F921FB61F921124BF
:103550008F939F93AF93BF938091B4029091B502E4
:10356000A091B602B091B7020196A11DB11D809342
:10357000B4029093B502A093B602B093B702BF9184
:10358000AF919F918F911F901FBE1F90189587E755
:1035900097E7809300089093010888E19AE00FB6BE
:1035A000F894A895809360000FBE90936000FFCFC1
:1035B00088E19AE00FB6F894A895809360000FBE5A
:1035C00090936000FFCF8EE1489B02C08150E1F7ED
:1035D000489BFECF0895589880E28A95F1F7589A53
:1035E0000895FC018BE08A95F1F798E020E080E0F7
:1035F00031E040E14A95F1F7880F489B02C08160B5
:10360000232742E04A95F1F7000040E14A95F1F79F
:10361000915079F790E19A95F1F799B132E03A95A6
:10362000F1F7000030E13A95F1F79170922720818F
:10363000920F90830895A1E0B0E0E0E2FBE1C1C702
:1036400019828C017C01E60EF11CBDDFCE010196D2
:10365000C8DFF80181938F01EE15FF05B1F781E016
:103660009981911180E02196E6E0C7C7509A589A57
:1036700008955098589AE89AE9E6F0E080818C7FA6
:10368000808308956150770B91E001C0990F6A958E
:10369000EAF7692F90E021E0611108C0911591F0DF
:1036A000589A80E28A95F1F758980895362F382372
:1036B00039F0589A922730E23A95F1F76695ECCFB7
:1036C0005898F9CF5898EDCFFF920F931F93CF934F
:1036D000DF93EC018C01060F111D8991F82E7BDF21
:1036E00068E08F2DCFDFC017D107B9F7CDB7DEB7B0
:1036F000E5E084C71F920F920FB60F9211240F932B
:103700001F932F933F934F935F936F937F938F9369
:103710009F93AF93BF93EF93FF93CF93DF930F925A
:10372000CDB7DEB719824FDFCE0101965ADF082FE1
:10373000069506950695282F22952570902F957051
:10374000920F292F237096959695920F9827977030
:103750008981892B09F055C0043008F052C080E1FE
:103760008A95F1F7589A509A82E08A95F1F700C04D
:10377000589888E0089F80011124D801AD5FBE4FA2
:103780001696ED91FD911897309791F06091A701F1
:103790007091A80114962D913D91260F371F159712
:1037A0008D919D91680F791F4C9113978C9109957C
:1037B000F801ED5FFE4F6381611549F02091A7018B
:1037C0003091A80184819581820F931F7DDF03DFF3
:1037D00080E18A95F1F758985098589A80E18A9537
:1037E000F1F7F801ED5FFE4F6081611549F020911E
:1037F000A7013091A80181819281820F931F1BDF65
:10380000E2DE0F90DF91CF91FF91EF91BF91AF91E9
:103810009F918F917F916F915F914F913F912F91E8
:103820001F910F910F900FBE0F901F9018950F933F
:103830001F93CF93DF93EC0104970CF05EC0F894D4
:10384000509A589885E08A95F1F700009C2F96953C
:1038500095708C2F8570980F892F8370969596950B
:10386000292F93E0CC0FDD1F9A95E1F7280F822FC7
:103870008C2B082FB0DE00C068E0802F03DF80E1D2
:103880008A95F1F75098589A489B30C087E090E0AD
:1038900048992EC0FE01ED5FFE4F6381611559F01E
:1038A0002091A7013091A80184819581820F931FF7
:1038B000C2DE8115F9F087DE80E28A95F1F758982B
:1038C000509A80E18A95F1F7CD5FDE4F68816115EE
:1038D00049F02091A7013091A80189819A81820F36
:1038E000931FF2DE78DE789481E008C000C0CCCF70
:1038F000019749F4509A589A789480E0DF91CF91DB
:103900001F910F91089500C0C3CF08959B01BA0184
:103910009091BC029430D9F48F708093E9009FEFAE
:103920008091E80085FD06C085ED8A95F1F70000DD
:103930009150B1F78091E80085FF09C040E050E068
:10394000C901BBD18091E8008E778093E80008958B
:1039500043E050E0BC0182E0D9CF46E050E0BC013A
:1039600082E0D4CFCF93DF93EC011BDD48E050E041
:10397000BE0181E0CBDF88E0FE01ACE8B2E001905F
:103980000D928A95E1F7DF91CF9108958091BB0266
:10399000811107C019D369D38091E20084608093BC
:1039A000E20008951092BB020895DEDC81E0EACCCB
:1039B0006091B80281E0611101C080E0C7CC9091B4
:1039C000BC0281E0943009F080E06091B802CACC7A
:1039D00042E061EC81E074D242E261EC82E070D2BC
:1039E0009091BC0281E0943009F080E06091B802CF
:1039F000A1CC8091BE02893081F148F4823009F473
:103A000096C0833009F457C0813041F008958A3060
:103A100009F480C08B3009F468C008958091BD021C
:103A2000813A09F047C08091E800877F8093E800E1
:103A30008091C1029091C202892B59F060E080E030
:103A400090E070E086D18091E8008B778093E80069
:103A5000089568E08CE892E0F4CF8091BD02813255
:103A600049F58091C1029091C202029718F58091A8
:103A7000E800877F8093E8008091E80082FF16C00D
:103A80002091F3008091F200922F029731F48091FF
:103A9000F100813011F0863019F48091F10084DC5E
:103AA0008091E8008B778093E8003EC28091BC0251
:103AB0008111E2CF08958091BD02813AD9F78091BA
:103AC000C1029091C202892BA9F78091E800877FFB
:103AD0008093E8008091E80080FFFCCF62DC809357
:103AE000F1008091E8008E77DECF8091BD028132B7
:103AF00009F78091C1029091C202892BD9F6809179
:103B0000E800877F8093E8000FD28091BF023ADC03
:103B10000C94B7068091BD02813261F68091E80075
:103B2000877F8093E80000D28091C0024BCC8091C7
:103B3000BD02813A09F0BECF8091E800877F809373
:103B4000E8008091E80080FFFCCF47DCC8CF84B755
:103B5000877F84BF0FB6F894A89580916000886134
:103B600080936000109260000FBE80E890E00FB676
:103B7000F89480936100909361000FBE01CC24D231
:103B800074D2E2EEF0E08081846080837894D1C4C6
:103B900085E291E0B0CA8091BC02853029F4809121
:103BA000BC02853011F0AACC08957DDC21DC8115A2
:103BB000B1F38091BA02811591F369D00E94B706E2
:103BC0008FEF99E628E1815090402040E1F700C056
:103BD0000000E5CF08959A014091C3025091C402BC
:103BE00000C0492F50E043305105D1F078F4413006
:103BF000510509F43DC04230510571F48BE390E06A
:103C00004EE253E0F901408351830895413251055A
:103C1000E9F04232510519F180E090E040E0F2CF46
:103C2000482F50E0813061F04230510561F0EAE206
:103C3000F3E04115510581F7849190E0AF01E2CFA7
:103C4000EAE1F3E0F9CFECEEF2E0F6CF6130710596
:103C5000A0F011F789E090E049E553E0D3CF61305F
:103C6000710580F0C9F68BE790E04BE753E0CACFCF
:103C700082E190E049E653E0C5CF89E090E040E47E
:103C800053E0C0CF84E490E046EF53E0BBCF80E147
:103C900089BD82E189BD09B400FEFDCF8091D800C5
:103CA0008F7D8093D8008091E00082608093E00057
:103CB0008091E00081FDFCCF0895AF92BF92CF923A
:103CC000DF92EF92FF921F93CF93DF937C01EB0182
:103CD0006A0149D1182F811122C0C114D10439F0D1
:103CE000F60180819181C81BD90BE80EF91EA12C29
:103CF000B12C2097A1F08091E80085FD20C0809133
:103D0000E8008E778093E800C114D10499F0F601A1
:103D1000808191818A0D9B1D8083918315E0812F85
:103D2000DF91CF911F91FF90EF90DF90CF90BF90E8
:103D3000AF90089518D18115F1F2182FF0CFF70147
:103D400081917F018093F10021978FEFA81AB80A23
:103D5000D0CFFC018091C3029091C40286179707CF
:103D600020F06115710561F0CB0140E0009771F41E
:103D700041110CC08091E80082FF36C080E00895B8
:103D80008091E8008E778093E800EECF2091BC020E
:103D90002115B1F12530B1F12091E80023FD2EC0AD
:103DA0002091E80022FDE6CF2091E80020FFDECF41
:103DB0004091F3002091F200342F009719F0283041
:103DC000310558F041E02830310509F040E02091FC
:103DD000E8002E772093E800C9CF41914093F1008D
:103DE00001972F5F3F4FE9CF8091BC02811541F0D1
:103DF000853041F08091E80083FFBCCF81E00895D9
:103E000082E0089583E00895FC018091C3029091BF
:103E1000C4028617970720F06115710561F0CB0188
:103E200040E0009771F441110CC08091E80082FFDE
:103E300037C080E008958091E8008E778093E80095
:103E4000EECF2091BC022115B9F12530B9F12091B6
:103E5000E80023FD2FC02091E80022FDE6CF20914D
:103E6000E80020FFDECF4091F3002091F200342FD4
:103E7000009719F02830310558F041E0283031051D
:103E800009F040E02091E8002E772093E800C9CFA8
:103E900044914093F100319601972F5F3F4FE8CF57
:103EA0008091BC02811541F0853041F08091E8009D
:103EB00083FFBBCF81E0089582E0089583E00895F9
:103EC000982F973028F08F708093E90081E0089553
:103ED0009093E900242F762F50E0981731F07091DD
:103EE000EC002091ED005091F00021FD02C09F5F99
:103EF000E8CF3091EB003E7F3093EB003091ED0046
:103F00003D7F3093ED003091EB0031603093EB005A
:103F10007093EC002093ED005093F0002091EE00A0
:103F200027FDE5CF80E008958091BD0287FF13C093
:103F30008091E80082FF06C08091E8008B77809333
:103F4000E80008958091BC028111F2CF089580911C
:103F5000BC028115D9F38091E80080FFF8CF8091F1
:103F6000E8008E77ECCF2091E4003091E50095E6F3
:103F7000A9012091EC00822F817020FF06C0809162
:103F8000E80080FF06C080E008952091E80022FD4F
:103F90001AC08091BC02811589F0853089F080912A
:103FA000EB0085FD0FC02091E4003091E500421741
:103FB0005307F9F29150E1F684E0089582E0089504
:103FC00083E0089581E008955FD066D0E0EEF0E0F0
:103FD000808181608083E8ED80818F77808319BC48
:103FE000A7EDB0E08C918E7F8C9380818F7E808353
:103FF0001092BB020895CF93DF9346D04DD0C8ED09
:10400000D0E088818F7788838881806888838881E1
:104010008F7D888319BC1092BC021092B802109256
:10402000BA021092B902E0EEF0E080818B7F8083CB
:1040300088818160888342E060E080E041DFE1EEDA
:10404000F0E080818E7F8083E2EE808181608083DA
:10405000808188608083E0EE80818E7F808388818C
:1040600080618883DF91CF910895E8EDF0E0808151
:104070008F7E8083E7ED80818160808384E082BFD2
:1040800081E08093BB02B7CFE8EDF0E080818E7FC6
:1040900080831092E20008951092DA001092E100FD
:1040A00008951F920F920FB60F9211242F933F93F2
:1040B0004F935F936F937F938F939F93AF93BF9330
:1040C000EF93FF938091E10082FF0AC08091E200AC
:1040D00082FF06C08091E1008B7F8093E10028D2AF
:1040E0008091DA0080FF18C08091D80080FF14C052
:1040F0008091DA008E7F8093DA008091D90080FF72
:104100008FC080E189BD82E189BD09B400FEFDCF89
:1041100081E08093BC023ADC8091E10080FF18C00E
:104120008091E20080FF14C08091E2008E7F809336
:10413000E2008091E20080618093E2008091D800EB
:1041400080628093D80019BC85E08093BC0230DC8B
:104150008091E10084FF28C08091E20084FF24C0A8
:1041600080E189BD82E189BD09B400FEFDCF809167
:10417000D8008F7D8093D8008091E1008F7E80935E
:10418000E1008091E2008F7E8093E2008091E20066
:1041900081608093E2008091B802811509F445C0E6
:1041A00084E08093BC020BDC8091E10083FF27C098
:1041B0008091E20083FF23C08091E100877F80939C
:1041C000E10082E08093BC021092B8028091E1008D
:1041D0008E7F8093E1008091E2008E7F8093E200E9
:1041E0008091E20080618093E20042E060E080E044
:1041F00067DE8091F00088608093F000D6DBFF914D
:10420000EF91BF91AF919F918F917F916F915F914E
:104210004F913F912F910F900FBE0F901F901895C7
:1042200019BC1092BC02BEDB77CF8091E30087FF00
:1042300002C083E0B6CF81E0B4CF1F920F920FB6D9
:104240000F9211241F932F933F934F935F936F937C
:104250007F938F939F93AF93BF93CF93DF93EF930E
:10426000FF93E9EEF0E080811091EC008F7010FB7D
:10427000112717F9182B1082C0EFD0E08881877FB3
:10428000888378941CD0E9EEF0E010828881886001
:1042900088831F701083FF91EF91DF91CF91BF91C1
:1042A000AF919F918F917F916F915F914F913F91CE
:1042B0002F911F910F900FBE0F901F901895AAE29B
:1042C000B0E0E4E6F1E280C18DEB92E0FC01019602
:1042D0002091F100208322E0853C9207B9F789DB29
:1042E0008091E80083FF37C08091BD029091BE02AB
:1042F0009A3088F5E92FF0E0EF51FC4D50C180383D
:1043000089F0823841F58091C1028F70873018F5AD
:104310008093E9008091EB0085FB882780F910925B
:10432000E90006C08091BA02880F9091B902892BEA
:104330009091E800977F9093E8008093F1001092AD
:10434000F1008091E8008E7722C0811115C0809124
:10435000BF02813001F18091E80083FF0AC08091A3
:10436000E800877F8093E8008091EB008062809373
:10437000EB00AA96E3E044C1823069F78091BF0266
:10438000811579F01092E9008091E800877F809391
:10439000E800CADDE0CF933009F080E08093BA02F4
:1043A000F1CF8091C1028F70282F2150263098F6CE
:1043B0008093E9002091EB0020FFE4CF933031F4AB
:1043C0008091EB0080628093EB00DCCF9091EB005A
:1043D00090619093EB0021E001C0220F8A95EAF7EB
:1043E0002093EA001092EA008091EB008860EBCF06
:1043F0008111B1CF8091BF028F77182F8091E30098
:104400008078812B8093E3008091E800877F809300
:10441000E8008ADD8091E80080FFFCCF8091E30016
:1044200080688093E30083E0111101C082E08093F3
:10443000BC0291CF8058823008F08DCF8091BF02AE
:104440009091C0028C3D23E0920789F583E08A8336
:104450008AE289834FB7F894DE01139620E03EE0AC
:1044600051E2E32FF0E050935700849120FF03C006
:1044700082958F703F5F8F708A30B8F0895C8D9322
:104480001D922F5F243169F74FBF8091E800877F2D
:104490008093E8006AE270E0CE0101965ADC8091D8
:1044A000E8008B778093E80056CF805DE8CF60917D
:1044B000C1027091C2029E012F5F3F4FA9018BDBA9
:1044C000BC01892B09F447CF9091E800977F909326
:1044D000E80089819A8198DCE2CF803809F03BCFEF
:1044E0008091E800877F8093E8008091B8028093F4
:1044F000F10027CF81112FCF9091BF02923008F0A9
:104500002ACF8091E800877F8093E8009093B802DB
:104510000BDD8091B802811529F084E08093BC0204
:1045200057DA19CF8091E30087FDF7CF81E0F6CF0E
:104530000895CF938091BC02811591F08091E9009C
:10454000C091EC008F70C0FBCC27C7F9C82B10922C
:10455000E9008091E80083FDB2DECF70C093E900EE
:10456000CF91089531DD1092BC0208958091E3004F
:1045700087FB882780F9089597FB072E16F400948F
:1045800006D077FD08D048D007FC05D03EF49095C2
:1045900081959F4F0895709561957F4F0895EE0F17
:1045A000FF1F0590F491E02D09942F923F924F92B6
:1045B0005F926F927F928F929F92AF92BF92CF92B3
:1045C000DF92EF92FF920F931F93CF93DF93CDB7BC
:1045D000DEB7CA1BDB0B0FB6F894DEBF0FBECDBF34
:1045E00009942A88398848885F846E847D848C8405
:1045F0009B84AA84B984C884DF80EE80FD800C810E
:104600001B81AA81B981CE0FD11D0FB6F894DEBFF0
:104610000FBECDBFED010895AA1BBB1B51E107C022
:10462000AA1FBB1FA617B70710F0A61BB70B881F42
:10463000991F5A95A9F780959095BC01CD010895D1
:10464000FB01DC0104C08D910190801921F44150DF
:104650005040C8F7881B990B0895FB01DC0102C08C
:1046600001900D9241505040D8F70895F999FECF2E
:1046700092BD81BDF89A992780B50895A8E1B0E070
:1046800042E050E020C0262FF999FECF92BD81BDB7
:10469000F89A019700B4021639F01FBA20BD0FB680
:1046A000F894FA9AF99A0FBE08950396272FECDF33
:1046B000EADF252FE9DF242FE7CF0196272FE4DF5C
:1046C000E2CFDC01CB01FC01F999FECF06C0F2BDBF
:1046D000E1BDF89A319600B40D9241505040B8F7C0
:1046E0000895F894FFCFEC04EC04230523057A0524
:1046F0009605140514059A050C0619061906781373
:104700006F137B136C13611361136C1361136113CB
:1047100097136113A2136113611361136113611382
:104720006C13611361136C136113891361136113AB
:10473000B713B713B713B713B713B713B713B71329
:10474000B7136413611378136B13081577151015DD
:10475000DA14DE141415E21418152415EE1470156D
:10476000F2142815F6142C155115FA143015581595
:10477000001536153E15E6141C15EA14201504150F
:104780003A15481561156E15D4140C157E151716BB
:104790001C161E162316331633163316331633160D
:1047A000331633163316251629162C1631164016D5
:1047B00046164A1656185C1847185018621868189A
:1047C0006E187F21A521AB21A521AB21F8211A224A
:0647D000AB216D227A22EC
:1047D60026020100000001000000000000000601A2
:1047E60000000004070000000000002808503C07F5
:1047F6001400000100DF19B21C851CAD1CA81CE2C8
:1048060000E900EA00B500B600B700CD008301CC90
:10481600008A019201940121022302240225022624
:104826000227022A02B300B4006F0070009F01CB7A
:10483600019F02A002E200E900EA00B500B600B757
:1048460000CD008301CC008A01920194012102234C
:104856000224022502260227022A02B300B4006FB0
:104866000070009F01CB019F02A002946697C63498
:0A48760035F6F731333236500200F8
:00000001FF
